:104200002000560065007200730069006F006E00A8
:1042100020003100330020006A0061006E0076004B
:1042200020003200300031003100200050006100D9
:1042300075006C0046006A0075006A006F0020007F
:104240003100320046003600380033005F00330092
:1042500065006D002E0043002000200020000000BB
:104260004100440043002000310038006200690032
:104270007400730020004D004300500033003400F0
:104280003200340020002000310037006200690055
:10429000740073000D000A004D0061007800690091
:1042A0003D00310033003100300037003100200084
:1042B000500074007300200070006F0075007200E1
:1042C000200032002C00300034003800200056005E
:1042D0006F006C00740073000D000A000000000005
:1042E000FF00FF00FF00FF00FF00FF00FF00FF00D6
:1042F000FF00FF00FF00FF00FF00FF00FF00FF00C6
:104300007000610075006C0066006A0075006A004C
:104310006F000000FF00FF00FF00FF00FF00FF0034
:1043200052005300320033003200200039003600C2
:10433000300030000000FF00FF00FF00FF00FF0022
:104340007200FF00FF00FF00FF00FF00FF00FF0002
:10435000FF00FF00FF00FF00FF00FF00FF00FF0065
:10436000FF00FF00FF00FF00FF00FF00FF00FF0055
:10437000FF00FF00FF00FF00FF00FF00FF00FF0045
:10438000FF00FF00FF00FF00FF00FF00FF00FF0035
:10439000FF00FF00FF00FF00FF00FF00FF00FF0025
:1043A000FF00FF00FF00FF00FF00FF00FF00FF0015
:1043B000FF00FF00FF00FF00FF00FF00FF00FF0005
:1043C000FF00FF00FF00FF00FF00FF00FF00FF00F5
:1043D000FF00FF00FF00FF00FF00FF00FF00FF00E5
:1043E000FF00FF00FF00FF00FF00FF00FF00FF00D5
:1043F000FF00FF00FF00FF00FF00FF00FF00FF00C5
:00000001FF
